:020000040800F2
:10000000F0050020C90000089D1800087D160008B2
:1000100000000000000000000000000000000000E0
:10002000000000000000000000000000A11800080F
:1000300000000000000000009F180008A31800083E
:10004000DB00000800000000DB000008DB00000807
:10005000DB000008DB000008DB000008DB00000814
:1000600000000000DB0000086502000875020008BF
:10007000DB000008DB000008DB00000800000000D7
:10008000DB0000080000000000000000DB000008AA
:1000900000000000DB000008DB000008DB000008B7
:1000A00000000000DB00000800000000711F0008D5
:1000B0000448854600F0A2F8004800476120000887
:1000C000C046C046F0050020044880470448004769
:1000D000FEE7FEE7FEE7FEE7FEE7FEE79B19000806
:1000E000B100000830B50B46014600202022012453
:1000F00009E00D46D5409D4205D31D469540491B5C
:100100002546954040191546521E002DF1DC30BDA4
:10011000F0B51FB40646002082B005464024019188
:1001200000901BE0019922460F46304600F020F86F
:10013000049A059B801A994110D31046194622460D
:1001400000F04BF8361A8F4101972246012000211A
:10015000009F00F042F838184D4100902046641E80
:100160000028DFDC019B00982946324607B0F0BD2D
:1001700010B5202A04DB0846203AD040002110BDEB
:100180000B46D340D0402024A21A91400843194680
:1001900010BD03460B439B0703D009E008C9121F9B
:1001A00008C0042AFAD203E00B780370401C491CF3
:1001B000521EF9D27047D2B201E00270401C491EB3
:1001C000FBD270470022F6E710B513460A460446F4
:1001D0001946FFF7F0FF204610BD10B5202A04DBBA
:1001E0000146203A9140002010BD914020239C1AE6
:1001F0000346E3401943904010BD0000064C012522
:10020000064E05E0E36807CC2B430C3C98471034BE
:10021000B442F7D3FFF750FF642400088424000899
:10022000417802780802104340BA704770B4FF2347
:100230004A1E1C4692B200290CD0084D084E017887
:10024000401C59406B5C6340745C1146521E92B274
:100250000029F4D11802204370BC70474C220008DA
:100260004C23000810B5024800F096F810BD0000BD
:100270004801002010B5024800F08EF810BD0000C3
:100280008C01002072B6FEE770B5044600F0E0FA7B
:100290001A4D0646E868C0070DD0601C08D0002C37
:1002A00004D000F0D5FA801BA04201D9032070BD14
:1002B000E868C007F1D1E868800601D52020E86031
:1002C000E868C00602D4E868400715D5E968002050
:1002D000CA060B4904D5C86902221043C861102020
:1002E000EA68520705D5CA6901231A43CA61042185
:1002F0000843E860012070BD002070BD002002406E
:10030000D0010020014620314A780023022A04D07F
:10031000042282630B700120704730B402681468B5
:100320000E25AC431460026814686408640014600D
:100330000125046C2A46C06BA24042604D700B70D0
:1003400030BC0020704770B50024014620314A7847
:10035000022A03D004218163012416E00268136895
:100360000E25AB431360026813685B085B001360E3
:100370000125036C2A469A40C36B5A604D700022D7
:100380000A70416B002900D08847204670BD806B01
:100390007047203040787047F0B4C16B0C6801683A
:1003A0000B680426056C3246AA40224210D05A0738
:1003B0000ED50A68920602D40A68B2430A60016C3C
:1003C0008E40C16B4E60C16A002935D1F0BC7047C8
:1003D0000227AF400246274001262032002F15D0C9
:1003E0009F0713D50B689B0604D40B680A24A3430C
:1003F0000B605670036C02219940C36B5960002159
:100400001170816A002917D1F0BC70470827AF40EE
:100410002742F9D01B07F7D50B680E24A3430B60C6
:10042000016C33468E40C16B4E6083635370002174
:100430001170016B0029E7D0F0BC0847002801D1FA
:100440000120704770B504460220254620356870AB
:10045000206802681049A3680A4061682669194348
:10046000E3683343194363691943A3691943E36993
:100470001943114301600949206840181421FFF70E
:1004800031FE800020640648E0630020A063012163
:100490006970287070BD00000FC0FFFFF8FFFDBF3E
:1004A00000000240F0B4044694462034227800252F
:1004B000012A0AD00127277066780022012E07D072
:1004C000227002252846F0BC7047F0BC022070471D
:1004D000022666708263026814686408640014600F
:1004E000046C3E46A640C46B624666600468636066
:1004F0004368102B03680AD099600168CA60C16A1A
:10050000002901680A6806D00E231A430AE09A609F
:100510000268D160F3E70A231A430A6001680A6897
:1005200004239A430A600068016839430160C9E7FF
:1005300070B5044600F08CF90546601C02D00448F2
:100540000078241800F084F9401BA042FAD370BD53
:1005500014000020F3B5054681B0012000902E481C
:10056000017E01290DD00121017628682B4C2C4EEB
:100570004027012808D02046FFF786FE002819D022
:1005800044E0022003B0F0BD2046FFF77DFE0028C6
:100590003CD12149C8613069042528433061306964
:1005A000384330612046FFF76FFE00903069A84362
:1005B00030612BE000210298C9430160A8686C6893
:1005C00080020019A04221D913490020C861306976
:1005D000022738433061746130694021084330613B
:1005E0000E48FFF751FE00903069B8433061009823
:1005F000002802D00298046008E00120800224183C
:10060000A868696880024018A042DDD8024900202D
:100610000876009803B0F0BDD001002050C3000060
:10062000002002400348016980221143016100203B
:100630007047000000200240F0B51FB405461D4879
:100640000024017E012907D0012606761A48FFF70B
:100650001BFE002803D027E0022005B0F0BD012DCD
:1006600002D0022D00D00425002D1DD9134E019873
:1006700061000F18220103990298FFF779FD0D4AD6
:100680000021D161316901221143316138800A486A
:10069000FFF7FAFD3169490849003161002803D1AB
:1006A000641CE4B2AC42E2D3024A0021117605B0E8
:1006B000F0BD0000D001002050C300000020024027
:1006C000064900200A69120607D5054A4A60054A0C
:1006D0004A600969090600D50120704700200240E0
:1006E00023016745AB89EFCD0B680022002B72D048
:1006F000F8B401270B6897403B406DD00C79A407F4
:10070000A40F012C01D0022C10D1856854000326BF
:10071000A640B543CE68A6402E43866044680D7956
:10072000BC43ED06ED0F9540254345600C79E4434D
:10073000A40708D0C56854000326A640B5438E68B8
:10074000A6402E43C6600C79A407A40F022C0CD13E
:10075000D408A40027183D6A5407E40E0F26A640CB
:10076000B5430E69A6402E433E6205685400032639
:10077000A640B5430E79B607B60FA6402E430660D5
:100780004C68A403A40F49D0284CA5690126354321
:10079000A561A469950834400094254CAD002F193B
:1007A000BD689407240F0F26A640B5430926F60618
:1007B000B04201D1002611E01E4EB04201D1012607
:1007C0000CE01D4EB04201D1022607E01B4EB042A4
:1007D00003D1032602E028E020E00526A6402E43B0
:1007E000BE60174D2C684E689C43F60300D51C4331
:1007F0002C606C684E689C43B60300D51C436C604B
:10080000AC684E689C43F60200D51C43AC60EC68B3
:100810004E689C43B60200D51C43EC600B68521C2A
:10082000D34000D065E7F8BC704770470010024025
:10083000000001400004004800080048000C004887
:1008400000040140002A01D0816170478162704735
:10085000014880687047000014000020002801D182
:100860000120704770B50446216816480860216869
:10087000154808602068616841602168A068886048
:10088000FFF7E6FF05462068C06840070ED0FFF777
:10089000DFFF401B272805D92068C068400701D02A
:1008A000032070BD2068C0684007F0D1206802694D
:1008B000E1688A4201D0016101E004490160002041
:1008C00070BD0000CCCC000055550000AAAA000065
:1008D000006802490160002070470000AAAA0000D9
:1008E00002488168027889188160704714000020EE
:1008F00010B506480168102211430160032000F082
:1009000007F800F027F8002010BD0000002002408A
:1009100070B504460D4D7D202978C000FFF7E2FB3D
:1009200001460B480068FFF7DDFB00F099FB00284B
:1009300009D1042C07D200222146401E00F02AF8DB
:1009400000206C6070BD012070BD0000140000200C
:1009500020000020084881B0816901221143816193
:10096000816911400091C26901040A43C261C069F2
:100970000840009001B0704700100240002805DBDD
:10098000C106C90E01208840014908607047000077
:1009900000E100E08207D30EFF229A408907090E8A
:1009A0009940002808DB830809489B001818036851
:1009B00093430B43036070470007000F0838830818
:1009C00004489B001818C36993430B43C3617047E5
:1009D00000E400E000ED00E0F8B504460068394EA0
:1009E000C0035AD5F0690025C00007D4F06931046E
:1009F0000843F061F0690840012500903248016821
:100A0000C90515D40068FF21013108432E4908604B
:100A1000FFF71EFF07462C480068C00508D4FFF703
:100A200017FFC01B642825D827480068C005F6D5E5
:100A3000306A03210902084021D062680A408242DC
:100A40001DD0306A326A8843012109040A433262A8
:100A5000326A8A4332623062C00710D0FFF7F8FE74
:100A60000746306A80070AD4FFF7F2FEC11B174819
:100A7000814201D90320F8BD306A8007F4D5306A7D
:100A8000032109028843616808433062002D04D0C5
:100A9000F069012109078843F0612078C00705D07B
:100AA000306BA1688008800008433063207880069E
:100AB00005D5306B10218843E1680843306300207E
:100AC000F8BD0000001002400070004088130000D4
:100AD000002801D101207047F8B504463E480D4674
:100AE0000068C007C00FA8420AD23B480168490805
:100AF0004900294301600068C007C00FA84250D1D7
:100B00002068364E81070CD5400704D57068072150
:100B10000902084370607068F0218843A1680843A7
:100B200070602078C0072CD0606801281BD0316825
:100B300002281CD0890734D57168890889000143CF
:100B40007160FFF785FE7168074662680C200140FE
:100B50009200914215D0FFF77BFEC11B20488142D5
:100B600008D90320F8BD316889031AD5E4E7890163
:100B700017D5E1E770680C21084061688900884258
:100B8000E9D115480168C907C90FA9420BD9016805
:100B900049084900294301600068C007C00FA84206
:100BA00001D00120F8BD2078400706D570680721E4
:100BB00009028843E1680843706000F027F8716813
:100BC000084A0906090F515CC8400749086003201C
:100BD000FFF79EFE0020F8BD0020024000100240FA
:100BE000881300004C240008200000200448054918
:100BF00000684968044A4905490F515CC84070477C
:100C000020000020001002405C24000810B514A051
:100C10000FC888B06C460FC415A00FC80FC4184A7F
:100C200053680C20194601401648042916D008299B
:100C300014D19902090F6C46645CD16A04AA0907B1
:100C4000090F525CD90305D500231946FFF760FA56
:100C5000214601E020460C4901F0DAF908B010BD48
:100C600002030405060708090A0B0C0D0E0F1010ED
:100C70000102030405060708090A0B0C0D0E0F10EC
:100C80000010024000127A0000093D00002801D146
:100C900001207047F8B504460078EE4DC00754D0E7
:100CA00068680007800F012807D068680007800F78
:100CB000022809D16868C00306D52868800344D596
:100CC0006068002874D040E0606801280CD00121E1
:100CD000890400280DD0052825D02A688810824371
:100CE0002A60286888430BE028680121090408432A
:100CF00006E028680122120490432860286888438F
:100D000028606068002812D0FFF7A2FD0646286818
:100D100080031AD4FFF79CFD801B642873D82868D1
:100D20008003F7D511E0286808432860DCE7FFF767
:100D30008FFD06462868800307D5FFF789FD801BD5
:100D4000642860D828688003F7D42078800741D5CC
:100D500068680007800F07D068680007800F0228C6
:100D600009D16868C00306D42868800718D5E068F0
:100D700001281DD114E0E0680028286819D001215D
:100D800008432860FFF764FD06462868800707D4FB
:100D9000FFF75EFD801B022835D828688007F7D54D
:100DA0002868F82188432169C9000843286011E0B8
:100DB0004CE1400840002860FFF74AFD06462868DD
:100DC000800707D5FFF744FD801B02281BD8286841
:100DD0008007F7D42078000727D5E0690028686AE3
:100DE00012D0012108436862FFF732FD0646686AA7
:100DF00080071AD4FFF72CFD801B022803D8686AED
:100E00008007F7D511E08BE0400840006862FFF7EB
:100E10001FFD0646686A800707D5FFF719FD801B8E
:100E200002287DD8686A8007F7D420780426400716
:100E3000002866DAE8690027C00007D4E869B1062F
:100E40000843E861E869084001270090824801688A
:100E5000C90515D40168801501437F480160FFF77B
:100E6000F7FC00907C480068C00509D4FFF7F0FC4F
:100E70000099401A64287DD877480068C005F5D5E8
:100E8000A06801280AD0002801D005281ED0286AB1
:100E9000400840002862286AB04302E0286A012125
:100EA00008432862A068002814D0FFF7D1FC009006
:100EB000286A80071ED4FFF7CBFC0099411A6748C7
:100EC000814257D8286A8007F5D513E0286A304355
:100ED0002862E3E7FFF7BCFC0090286A800709D589
:100EE000FFF7B6FC0099411A5C48814242D8286A53
:100EF0008007F5D4002F04D0E86901210907884351
:100F0000E8612078C0061BD56069012834D0401DF7
:100F1000686B4ED030436863686B4008400000E067
:100F200028E06863FFF794FC0646686B800707D5E6
:100F3000FFF78EFC801B02281CD8686B8007F7D453
:100F4000206A002868D069680907890F022968D0DB
:100F500001263606022828682ED0B0432860FFF705
:100F600077FC04462868800172D5FFF771FC001BEE
:100F7000022852D90320F8BD686B30436863686B60
:100F8000012108436863FFF763FC0646686B80072E
:100F900007D4FFF75DFC801B0228EBD8686B800745
:100FA000F7D5686BF8218843A169C90008436863D5
:100FB000C6E7B0436863F4E7B0432860FFF748FC36
:100FC00007462868800107D5FFF742FCC01B0228AE
:100FD000D0D828688001F7D4E86AE16A00090001E6
:100FE0000843E862616AA06A084369683D22120406
:100FF000914308436860286830432860FFF728FC65
:1010000004462868800123D4FFF722FC001B022835
:10101000B0D828688001F7D51AE028688001A4D4E8
:1010200016E00128A7D06868E96A01221204636A01
:1010300002409A420AD10907E26A090F914205D19A
:101040000F2189040840A16A884201D00120F8BD1F
:101050000020F8BD0010024000700040881300001E
:101060000B4910B4401E884202D910BC01207047C1
:101070000849486108480722C3691B021B0A4C043F
:101080002343C361002088610A6110BC70470000DF
:10109000FFFFFF0000E000E004ED00E07047F8B55E
:1010A000816F0446C66F00688268254612061027C5
:1010B0008035002A26DA212924D1EFF3108101227C
:1010C00082F31088826880239A43826081F31088BB
:1010D000E06E002808D0FFF715F9002804D0E06E74
:1010E000FFF755F920282FD0EFF31081012080F36E
:1010F000108820680268C0239A43026081F3108838
:101100002020A0672068816849061BD5222E19D1AE
:10111000EFF31081012282F31088826840239A4302
:10112000826081F31088206F002808D0FFF7EAF86A
:10113000002804D0206FFFF72AF9202804D0204689
:1011400000F080FD0020F8BD2F600320F8BD70473F
:10115000F8B502680446D069116896689F4B054649
:101160001D402023002D76D0F7079D4DFF0FBC4674
:101170000D402F436ED02546C7078035002F06D07F
:10118000CF0504D5012717622A683A432A608207EF
:1011900008D5F20706D0276802223A622A68042797
:1011A0003A432A60420708D5F20706D0266804228F
:1011B00032622A68022632432A6002070AD50A46AA
:1011C0001A406646324305D02668082232622E68ED
:1011D00016432E60020508D54A0106D5012226686D
:1011E000D20232622A681A432A602A68002A2FD063
:1011F000800606D5880604D5616E002901D02046F8
:101200008847286821688968490602D4282108424D
:101210002DD0204600F016FD20688168490622D5B1
:10122000EFF31081012282F31088836840229343F8
:10123000836081F31088206F002814D069494163CE
:10124000206FFFF780F8002802D0206F416B88479D
:10125000F8BD00E011E085060FD58D060DD5616E55
:1012600000297CD1F8BD2046FFF771FFF8BD20466C
:10127000FFF76DFF00202860F8BD256E012D6FD1AE
:10128000C5066DD5CD066BD510271762206881681D
:10129000254649064035002948DA226F1168496819
:1012A0000904090CE8D02E8B8E42E5D96983916937
:1012B000202933D0EFF31081012282F310880268D5
:1012C0003E01B243026081F31088EFF310810120E8
:1012D00080F310882068826852085200826081F38F
:1012E0001088EFF31081012080F310882068866851
:1012F00040229643866081F31088E36700202066D1
:10130000EFF31081012080F3108820680368BB434D
:10131000036081F31088206FFEF7F4FF288B698B40
:10132000401A81B22046FFF7B9FEF8BD298B6A8BBF
:10133000891A6A8B89B2002AF7D00029F5D0EFF319
:101340001082012585F310880568FF262136B543F4
:10135000056082F31088EFF31082012001E023E0A2
:101360001BE080F31088206885686D086D0085603B
:1013700082F31088E36700202066EFF31082606636
:10138000012080F3108820680368BB43036082F368
:1013900010882046FFF782FEF8BD050607D50D062A
:1013A00005D5A16E0029F7D020468847F8BD400634
:1013B000FCD54806FAD52046EFF31081012484F3CA
:1013C000108814684025AC43146081F3108883674B
:1013D0000021816600F050F9F8BD00000F08000000
:1013E00020010004CD1A0008002801D10120704717
:1013F00010B50446806F002805D1002174200155E6
:10140000204600F027F82420A067206801684908DA
:1014100049000160204600F045FC012818D0606AB0
:10142000002802D0204600F0B9FA20684168012265
:10143000D202914341602068816808229143816013
:1014400020680168012211430160204600F00CFB76
:1014500010BD0000F0B587B000240546009401944B
:101460000294039404940068314988425DD1314864
:101470008269012189030A43826182690A400592D7
:101480004269C9000A43426140690840059003204F
:10149000400200900220019003200390012004905C
:1014A00009206946C006FFF71FF9244E80277460A3
:1014B000B46034617461F7601F48B46130608014B7
:1014C000F0613046FEF7BAFF002801D0FEF7DAFEE1
:1014D0002E6775621B4E1A483060B46034617461C7
:1014E000F7601020B46170600002F0613046FEF7D2
:1014F000A5FF002801D0FEF7C5FE1348016842157C
:1015000011430160EE66002211461B207562FFF751
:1015100041FA1B20FFF732FA0C4B186802681021C1
:101520000A43026019685020086207B0F0BD00004D
:101530000038014000100240300002404801002005
:10154000440002408C01002000000140C400002043
:1015500070B5C36F202B2BD100290BD0002A09D0E6
:10156000012483682403A34206D10369002B03D11D
:10157000CB0701D0012070BD034660331C7D012CD8
:1015800016D001241C750023036603685C682402DE
:101590000BD5EFF31084012585F310881D68012613
:1015A000B60635431D6084F3108800F00BFC70BD57
:1015B000022070BD70477047F8B50446806F202840
:1015C00052D100290BD0002A09D00123A0681B03A7
:1015D000984206D12069002803D1C80701D0012014
:1015E000F8BD25466035287D01283DD001202875AD
:1015F00020464030E164028242820027264680363F
:1016000037602120A067E06E00281BD01749816257
:10161000E16E1748C862E16E16480863E06E134633
:1016200047632068E16C283084466246E06EFEF72E
:1016300039FF002806D0102030602F752020A067C9
:101640000120F8BD2168402008622F75EFF310815A
:10165000012080F310882068826880231A4382600A
:1016600081F310880020F8BD0220F8BDF11B0008AE
:101670003B1C0008E11A000870477047FEE70000B5
:10168000F8B53B4E301DFEF7CBFD04B2B01CFEF7A3
:10169000C7FD054606213046FEF7C8FD0246354F18
:1016A0000020315C3954401CC0B20628F9D3110A1D
:1016B000D0B2B971304AF8710F2D06D0FF23F5333F
:1016C000042D2BD0052D3AD04CE0B379994249D165
:1016D000F179884246D1601EF6280ED8D4800120C8
:1016E00080F3108800F07AFD002838D13078002887
:1016F00035D0082000F052FD31E0FF2038717871BC
:1017000006211B48FEF792FD010AB971F871307885
:10171000002827D0082000F041FD23E0B579A94238
:1017200020D1F17988421DD19C421BDB54800120DD
:1017300080F3108800F052FD0028DAD00FE0B57970
:10174000A9420FD1F17988420CD19C420ADB9480E6
:10175000012080F3108800F041FD0028C9D000204E
:1017600080F3108820210248FEF72CFDF8BD000010
:1017700064000020440000200000002008B50C4850
:1017800041690122114341614069012110400090EB
:1017900000220A20FFF7FEF80A20FFF7EFF80022E8
:1017A00001210B20FFF7F6F80B20FFF7E7F808BD43
:1017B0000010024070B586B000241C4800940194CB
:1017C0000294039404944269012189050A43426109
:1017D00042690A400592426949110A4342614069DF
:1017E00009260840F60605900022E8213046FFF75A
:1017F00029F8012210213046FFF724F8C820009074
:10180000022002900320012503900195694630468D
:10181000FEF76AFF30200090019569460395029417
:101820003046FEF761FF06B070BD000000100240B8
:1018300010B5094807490160062141600749C160A8
:1018400007498160FFF70AF8002801D0FEF71AFD6A
:1018500010BD000000300040B4000020FF0F000069
:10186000B80B000010B50C480A4901604B21C901B2
:10187000416000218160C16001618161C1610C2210
:10188000016242614162FFF7AFFD002801D0FEF71F
:10189000F9FC10BD00380140C4000020FEE770478D
:1018A000704710B500F004F8FFF71AF810BD0000FB
:1018B00030B4194B58680124002804D05868401EE1
:1018C000586000D11C70154D00210C204843401970
:1018D0004268002A09D04268521E426005D1447015
:1018E0000278012A01D182684260491CC9B20429E8
:1018F000EBD39868401C98609868094A0021904290
:1019000000D199605878401CC0B258700A2800D3A2
:10191000597030BC7047000008000020840000208F
:10192000FFFFFF7F70B594B00024059404940F94DA
:10193000092002250E9400901394E8030294039466
:10194000069409900B940C940D94012600011094B8
:10195000119412940A900196079608956846FFF72D
:1019600095F9002801D072B6FEE707200C900E947E
:1019700001210D950F940CA8FFF7AAF8002801D0BB
:1019800072B6FEE710A810961294FFF725F800280B
:1019900001D072B6FEE714B070BD704710B4818CF0
:1019A000C90707D001684A6801235B049A43836A28
:1019B0001A434A60818C890707D501684A68012368
:1019C0001B049A43C36A1A434A60818C490707D5AE
:1019D00001684A6801239B049A43036B1A434A60D7
:1019E000818C090707D501684A680123DB039A4304
:1019F000436B1A434A60818CC90607D501688A681F
:101A000001231B039A43836B1A438A60818C8906E6
:101A100007D501688A6801235B039A43C36B1A43A5
:101A20008A60818C490612D501684B680122120533
:101A3000046C934323434B60016C914207D10168CE
:101A40004A6803235B059A43436C1A434A60818CBE
:101A5000090607D501684A680123DB04806C9A43B4
:101A600002434A6010BC7047F8B504460025803038
:101A70000560FEF7EDFE074620680068124E00077D
:101A800009D501213B46002249052046009600F079
:101A9000F3F900280DD12068006840070BD501211B
:101AA0003B46002289052046009600F0E5F9002813
:101AB00001D00320F8BD2020A067E06725666034D0
:101AC00025750020F8BD0000FFFFFF0110B5406A3A
:101AD0000022014640314A834A82FFF738FB10BD9D
:101AE00070B5446AA06FE26F216889680023090617
:101AF000002911DA21280FD152200353EFF310816E
:101B0000012080F3108820680568C026B543056071
:101B100081F310882020A06720688068400606D5E1
:101B2000222A04D15A200353204600F08BF8204685
:101B3000803001681022114301602046FFF707FB47
:101B400070BD10B501468969406A202937D000224E
:101B50005A210A52EFF31082012181F310880168A3
:101B60000B68FF240134A3430B6082F31088EFF36A
:101B70001082012181F3108801688B685B085B008B
:101B80008B6082F31088EFF31082012181F31088BB
:101B900001688B684024A3438B6082F31088202166
:101BA000C167016E01290AD1EFF3108281F3108819
:101BB00001680B681024A3430B6082F31088016E48
:101BC000012902D0FFF7F6FC10BD5821095AFFF792
:101BD00065FA10BD10B5406A016E012902D0FFF709
:101BE000EAFC10BD5821095A4908FFF757FA10BD01
:101BF00010B501468969406A20291BD00022522174
:101C00000A52EFF31082012181F3108801688B687A
:101C10008024A3438B6082F31088EFF310810122AC
:101C200082F310880068026840231A43026081F33F
:101C3000108810BDFFF720FD10BD10B5406AFFF7FA
:101C40001CFD10BD10B4EFF31082012181F3108848
:101C500001680B68FF242134A3430B6082F31088D2
:101C6000EFF31082012181F3108801688B685B0813
:101C70005B008B6082F31088016E01290AD1EFF3BB
:101C8000108281F3108801680B681024A3430B6055
:101C900082F310882021C16700210166416610BCD3
:101CA0007047000070B5044681680069E26901432D
:101CB0006069002510430143206802683C4B1A40CC
:101CC0000A43026020684168032212039143E268DC
:101CD00011434160216AA0690143206882680B2397
:101CE0001B029A430A4382603248006B8007800FD0
:101CF00006D0012816D0022816D0032810D01020B4
:101D00000122E369D2032C492C4E93422AD10028A8
:101D10000CD002280DD004280DD008283ED10EE0AA
:101D20000220EDE70420EBE70820E9E7FEF75EFF7D
:101D300003E00A4603E0FEF769FF020032D0616863
:101D400050004A088018FEF7CDF980B201461039DC
:101D5000B14223D81A4901400007420F20680A43C4
:101D6000C2601FE0002806D0022807D0042807D050
:101D7000082813D108E0FEF739FF03E00A4603E024
:101D8000FEF744FF02000DD0616848088018FEF796
:101D9000A9F980B201461039B14201D9012501E00B
:101DA0002168C86000206066A066284670BD0000FB
:101DB000F369FFFF0010024000127A00EFFF0000FD
:101DC000F0FF0000F8B50446416540300027264684
:101DD0000283803637602220E0672546206F603519
:101DE00000281BD021498162216F2148C862216FE0
:101DF00020480863206F13464763606D216884465E
:101E000062462431206FFEF74DFB002806D01020DB
:101E100030602F752020E0670120F8BD2F75EFF3AB
:101E20001081012080F3108820680268FF230133AD
:101E30001A43026081F31088EFF31081012080F3D0
:101E400010882068836801221343836081F310881F
:101E5000EFF3108182F310882068826840231A43D0
:101E6000826081F310880020F8BD0000431B000849
:101E7000D51B0008E11A0008FFB50446006881B0D0
:101E80000E460A9DC1691746304688433FD0002060
:101E9000B84268D1204660300090681C5BD0FEF7E5
:101EA000D7FC0499401AA84233D8002D31D02068BD
:101EB000016849074FD5C069C04300054BD40120D4
:101EC0002168C0020862EFF31081012080F31088BE
:101ED00020680268FF23A1339A43026081F31088CF
:101EE000EFF31081012080F3108820688268520887
:101EF0005200826081F310882020A067E067803460
:101F00002060009900200875032005B0F0BD012075
:101F1000BEE7EFF31081012080F31088206802688B
:101F2000FF23A1339A43026081F31088EFF31081FD
:101F3000012080F310882068826852085200826075
:101F400081F310882020A067E067009900200875C1
:101F5000032005B0F0BD2068C1693046884305D034
:101F60000020B84299D0002005B0F0BD0120F8E76C
:101F700010B51148FFF7ECF80F480068C169C94374
:101F8000C90618D4102101620B48FFF788F80B48E6
:101F9000017800290AD10A49096849682022511AA2
:101FA000CAB2027007490848FEF7F3F82022054933
:101FB0000148FFF7CDFA10BDC4000020000000204A
:101FC00048010020240000206400002010B50E48C5
:101FD0000E4C02784178E388204600789A4201D17D
:101FE000082802D0002A05D00AE0032908D00629D3
:101FF00006D103E0082803D1062901D1FFF740FBF1
:102000000020207010BD00006400002000000020AF
:10201000F0B4040C8BB2264682B25E430D0C10461F
:10202000370C5843360480190021794116466E4317
:10203000370C36048019794126466E438919F0BC65
:10204000704702E008C8121F08C1002AFAD1704781
:102050007047002001E001C1121F002AFBD1704728
:10206000FEF746FCFFF75EFCFFF7A4FBFFF786FBDD
:10207000FFF7F8FBFFF7DCFB3F4B404A188840496D
:102080001080002801D0884201D10120108058889A
:102090003C4D7D2212012880002801D0884200D1C9
:1020A0002A809888384E0028308001D0884200D19C
:1020B00032803648FEF70CFC3548FEF7F0FF202250
:1020C00034493348FFF744FA0924E406002280210A
:1020D0002046FEF7B7FB002240212046FEF7B2FB68
:1020E00027462D4C2948FEF7F3FB002210213846E5
:1020F000FEF7A8FB012280213846FEF7A3FB012250
:1021000008213846FEF79EFB2888FEF711FA0022C8
:1021100080213846FEF796FB002208213846FEF75C
:1021200091FB6420FEF704FA012210213846FEF7E5
:1021300089FB012240213846FEF784FB002208215A
:102140003846FEF77FFB3088FEF7F2F90022402187
:102150003846FEF777FB012208213846FEF772FB6E
:102160006420FEF7E5F920780028BBD0FFF72EFFAA
:1021700000202070B6E70000003C000806000020A8
:10218000FFFF00000200002004000020B400002037
:10219000C4000020240000200000002070B50924A5
:1021A0000546E406012220212046FEF74BFB2A4685
:1021B00007490848FFF700FA0748FEF7EAF8012840
:1021C000FAD1002220212046FEF73CFB70BD000022
:1021D00044000020C40000208C01002010B586B00F
:1021E0000020009001900290164C0120039404906E
:1021F000FEF766FA05A902A8FEF7ACF9002802D09E
:10220000012006B010BD104A6946D0880870000A47
:10221000487050888870000AC87090880871000A59
:10222000487121460320019B009AFEF705FA002819
:1022300002D0032006B010BDFEF7F4F9002006B06E
:1022400010BD0000003C00080000002000C18140DB
:1022500001C0804101C0804100C1814001C0804176
:1022600000C1814000C1814001C0804101C0804166
:1022700000C1814000C1814001C0804100C1814056
:1022800001C0804101C0804100C1814001C0804146
:1022900000C1814000C1814001C0804100C1814036
:1022A00001C0804101C0804100C1814000C1814026
:1022B00001C0804101C0804100C1814001C0804116
:1022C00000C1814000C1814001C0804101C0804106
:1022D00000C1814000C1814001C0804100C18140F6
:1022E00001C0804101C0804100C1814000C18140E6
:1022F00001C0804101C0804100C1814001C08041D6
:1023000000C1814000C1814001C0804100C18140C5
:1023100001C0804101C0804100C1814001C08041B5
:1023200000C1814000C1814001C0804101C08041A5
:1023300000C1814000C1814001C0804100C1814095
:1023400001C0804101C0804100C1814000C0C10185
:10235000C30302C2C60607C705C5C404CC0C0DCD15
:102360000FCFCE0E0ACACB0BC90908C8D81819D985
:102370001BDBDA1A1EDEDF1FDD1D1CDC14D4D515B5
:10238000D71716D6D21213D311D1D010F03031F1A5
:1023900033F3F23236F6F737F53534F43CFCFD3DD5
:1023A000FF3F3EFEFA3A3BFB39F9F83828E8E929C5
:1023B000EB2B2AEAEE2E2FEF2DEDEC2CE42425E575
:1023C00027E7E62622E2E323E12120E0A06061A1E5
:1023D00063A3A26266A6A767A56564A46CACAD6D95
:1023E000AF6F6EAEAA6A6BAB69A9A86878B8B97905
:1023F000BB7B7ABABE7E7FBF7DBDBC7CB47475B535
:1024000077B7B67672B2B373B17170B05090915124
:102410009353529296565797559594549C5C5D9D54
:102420005F9F9E5E5A9A9B5B995958988848498944
:102430004B8B8A4A4E8E8F4F8D4D4C8C44848545F4
:1024400087474686824243834181804000000000E6
:102450000000000001020304060708090000000054
:10246000010203048424000800000020240000006E
:1024700042200008A824000824000020CC05000009
:10248000522000080000E803E803010000000000FB
:102490000000000000000000010000000400000037
:0824A0000000000000127A00A8
:04000005080000B13E
:00000001FF
